:1000000000308A00972A0000FF00030E8301A10040
:100010000A08A0008A010408A2007708A300780853
:10002000A4007908A5007A08A6007B08A70083131E
:1000300083128B1E1D280B193028220884002308E8
:10004000F7002408F8002508F9002608FA00270818
:10005000FB0020088A00210E8300FF0E7F0E09009E
:100060008A110A123B290A108A100A1182070034E9
:1000700000340634403420340134FF343F34ED344E
:1000800009342D341234DB34243400340134313457
:10009000003407340034C0343F34C03409340034F1
:1000A0001034C034003400344034003412343F344F
:1000B000123400340934DB3400348F340034E63435
:1000C000003469340434FD34003401341234FF3414
:1000D0000034E734003400341C340034233400345A
:1000E0000634C834003400343034A3340834BB340C
:1000F0000134F7340034BF34003439340034DE3492
:1001000000347934003471340034BD340034F634B2
:100110000034093409341E34003470340634383461
:10012000003436342234363424343F340034F3344B
:1001300000343F340434F3340434ED3400340134F7
:1001400009343E340034303412343634143400343C
:10015000363400342A340934123460340034003424
:10016000243482340034003422340834003400341F
:100170002034F7340034BF34003439340034DE34F2
:1001800000347934003471340034BD340034F63432
:100190000034093409341E340034703406343834E1
:1001A000003436342234363424343F340034F334CB
:1001B00000343F340434F3340434ED340034013477
:1001C00009343E34003430341234363414340034BC
:1001D000363400342A3409341234403406340034BE
:1001E000093480343034C03412340A108A100A11B1
:1001F000FC3E03188A0A8200523465346134643448
:100200007934203474346F34203464346934733472
:1002100070346C3461347934203432342E340A34FE
:100220000D34003494138C11430893000230941B56
:1002300020298C1D192900308316111B01308312CF
:10024000F80000348D1194138316111483128D1944
:100250002229941B2229831611182C298312410864
:10026000C30012214208C30012218316111511196F
:10027000372983120034B00BC629A908031D83292E
:100280002A08B8003808B90039081F3C03185C294F
:1002900039087E3C031C5C292030B9020310390D5B
:1002A000F700BA003A0A3320FA003A083320F8007F
:1002B0007A08F9005F295F290030F800F900790811
:1002C000BA007808B9007908BC007808BB003B0880
:1002D000FF3ABD003C08BE004030C1003D08C200EE
:1002E00022213C08BD00BE013C08FF3ABF003E0889
:1002F000C0004230C1003F08C20022217F3086008A
:100300000130A900C4292B08B8003808B900390801
:100310001F3C03189F2939087E3C031C9F2920306D
:10032000B9020310390DF700BA003A0A3320FA0077
:100330003A083320F8007A08F900A229A2290030EF
:10034000F800F9007908BA007808B9007908BC000B
:100350007808BB003B08FF3ABD003C08BE004030B7
:10036000C1003D08C20022213C08BD00BE013C087E
:10037000FF3ABF003E08C0004230C1003F08C20043
:100380002221BF308600A9013230B0008B160B113C
:100390008A110A121D28B2013208013C031CD62919
:1003A0002C30320784008001B20ACC29AE01AF01A3
:1003B0008A110A12C92AA8132808831687008312F3
:1003C00087130830F800000000000000F817F72934
:1003D000F813B40C03188717031C87137817F72931
:1003E0007813F80BE9290000000000008717A730F8
:1003F0008400840BF9290000F81BE829781BF029F8
:1004000000340830F7002817280883168700831265
:10041000071B082AB201F7171B2AF7131B2A031020
:10042000071B0314B20C77171B2A7713F70B0F2A3D
:100430003208F800272AA730F71B2D30F800F80BF8
:100440001F2A0000F71B0D2A771B152A0F2A0034DC
:10045000B31B3A2A0F30F700320EF7050A30770245
:100460000318352A3030F707372A3308F70777089B
:10047000B400DB210F30B2050A3032020318422AE1
:100480003030442AB3133308B2073208B400DB21FA
:100490008A110A12EB2A2E08B5003308B600360876
:1004A0003507B700013C0318572A0230B702370856
:1004B000F8007808B4002C30340784000008F800F5
:1004C00000343208B3002C302F078400330880003A
:1004D000AF0A2F08023C0319AF01B3014B22780881
:1004E000AA000130B3004B227808AB00AB08031917
:1004F000882A2F082E020319862AAE0A2E08023CEB
:100500000319AE010130F800882A882A0030F8006B
:100510002A08B400DB212B08B400DB210A30B40028
:10052000DB210D30B400DB218A110A12F42A840188
:100530001F308305073083169F00FF308312A80009
:10054000A81328088316870083128717A815280880
:1005500083168700831228162808831687003130F7
:1005600093002830831294008316941714130130DB
:100570008312A900AA01AB016430B00083160912EE
:100580000108C039013881008601FF3083128600DE
:10059000CB29B2013208F520B20AB400DB211530B4
:1005A0003202031DCA2A01228B16C0308B0401229D
:1005B0007808B1003108B400DB212030B400DB2121
:1005C0003D30B400DB212030B400DB213108B20023
:1005D0003730B300282A0A30B400DB210D30B400D4
:0C05E000DB213108B200612AD72A630039
:02400E007A3FF7
:00000001FF
